:020000040000FA
:02000000EE28E8
:080008008E00030E8D00803014
:100010008107A620B4208030180203190617980A19
:100020009808031D1B280613990A3C301902031D6A
:100030001B289901C22023200B111E280D0E8300BE
:100040008E0E0E0E09008C03031D282804308C0030
:1000500001300C02031D31280E3085000F0893007B
:100060004C2802300C02031D3A280D308500100880
:1000700093004C2803300C02031D43280B308500ED
:10008000110893004C2804300C02031D4C28073043
:100090008500120893004C2800301302031D5528D8
:1000A0000611861106128612080001301302031D84
:1000B0005E28061586110612861208000230130209
:1000C000031D6728061186150612861208000330E4
:1000D0001302031D702806158615061286120800E5
:1000E00004301302031D79280611861106168612A4
:1000F000080005301302031D822806158611061616
:100100008612080006301302031D8B28061186157F
:1001100006168612080007301302031D94280615E0
:10012000861506168612080008301302031D9D2846
:100130000611861106128616080009301302031DE7
:100140000800061586110612861608001518AE2836
:100150000618080015143230960008009603031D97
:1001600008001510E12008001418BC2886180800A3
:1001700014143230970008009703031D0800141070
:10018000CE200800920A0A301202031D08009201D4
:10019000910A06301102031D08009101033010027C
:1001A000031DD92802300F02031DD92890018F01A9
:1001B0000800900A0A301002031D080090018F0AFF
:1001C0000800920A0A301202031D08009201910AE7
:1001D00006301102031D08009101080083128501F9
:1001E0008601831628308100103085008330860018
:1001F0008312A0308B00850181018F019001910154
:10020000920193019801990104308C0095019401A9
:0A0210003230960097000C290C29EB
:02400E00F23F7F
:00000001FF
